:0D01F900020C0000010810010B00012000A5
:03000B00020016DA
:10001600C0E0758ADC758C0B200309300104C2929E
:100026008002D292E508700F850C09850D0AF50C41
:0C003600F50DB2927508101508D0E032EC
:03000300020042B6
:10004200C0E0C0D0C000C001C0027A0079007800D0
:10005200E5112401F511EA3510F510E9350FF50F18
:10006200E8350EF50E050DE50D7002050CD002D037
:0800720001D000D0D0D0E03233
:0300130002007A6E
:09007A00C0D0A2B39200D0D03234
:080083003099FDC2998F99220A
:08008B003098FDC298AF9922E4
:10009300C2B4D2B3D2B7D292C290C291C203C20841
:1000A300759850438921758DFDD28ED299C298D20D
:1000B3008CD2AFD2A9D2A8D2AAD288D28A2098034E
:1000C3000201BEC298AF99EF12030C00ED0100F4D8
:1000D30002012A0301570400F90501500601010832
:1000E30001090901200A000001BED201C203020175
:1000F300BEC2010201BEAF201200830201BE7F080F
:100103001200830201BE7F0C1200837F2212008340
:100113007F381200837F4E1200830201BED2037F19
:100123000A1200830201BE850912850A13AE12AFBB
:10013300137C007DFF120293120083AE12AF137C77
:10014300007DFF120293AF05120083806E12008BB5
:100153008F208067851117851016850F15850E145E
:10016300751100751000750F00750E00AF17AE16F0
:10017300AD15AC1478101202F98E128F137C007D2A
:10018300FF120293120083AE12AF137C007DFF12A5
:100193000293AF05120083851612851713AE12AFB3
:1001A300137C007DFF120293120083AE12AF137C07
:1001B300007DFF120293AF05120083A2B792027F64
:1001C300887E137D007C00AB11AA10A90FA80ED363
:1001D3001202E84005200302C201A2B392003003D9
:1001E30007A2B392B40200C0300105C2B40200C03A
:0501F300D2B40200C0BF
:0101F80022E4
:03000000020207F2
:0C020700787FE4F6D8FD75812102024EDC
:10029300BC000BBE0029EF8DF084FFADF022E4CC4F
:1002A300F875F008EF2FFFEE33FEEC33FCEE9DEC18
:1002B300984005FCEE9DFE0FD5F0E9E4CEFD22ED5E
:1002C300F8F5F0EE8420D21CFEADF075F008EF2FA8
:1002D300FFED33FD4007985006D5F0F222C398FD99
:0502E3000FD5F0EA2236
:1002E800EB9FF5F0EA9E42F0E99D42F0E89C45F06C
:0102F80022E3
:1002F900E8600FECC313FCED13FDEE13FEEF13FFE3
:03030900D8F12206
:10030C00D083D082F8E4937012740193700DA3A380
:10031C0093F8740193F5828883E473740293686094
:06032C00EFA3A3A380DF94
:10021300020093E493A3F8E493A34003F68001F26E
:1002230008DFF48029E493A3F85407240CC8C333EC
:10023300C4540F4420C8834004F456800146F6DFBB
:10024300E4800B01020408102040809001F9E47E51
:10025300019360BCA3FF543F30E509541FFEE493B0
:10026300A360010ECF54C025E060A840B8E493A377
:10027300FAE493A3F8E493A3C8C582C8CAC583CAA2
:10028300F0A3C8C582C8CAC583CADFE9DEE780BE5A
:0102060000F7
:00000001FF
